:10000000830100308A0004288301292B8312900089
:10001000911B112811088A001008900A0319910AEF
:1000200082008313111883171008900A84000008B7
:100030000800483465346C346C346F343A342034FE
:0200400000348A
:1006160083128514013083121C2B83128C00043044
:100626008D00FA3083121C238D0B142B8C0B122B8E
:10063600080083128C0004308D0053308E008E0B20
:10064600222B8D0B202B8C0B1E2B0800831685016D
:100656000130860083128501860183120B2319302F
:100666008C0000308D0039234C23372B432B0D088B
:1006760091000C088C0A03198D0A062083128B231D
:1006860083120D0891000C08062000380319080093
:100696003A2B83128C0106184E2B29308D008D0BB8
:1006A600522B06180C1421308D008D0B582B061872
:1006B6008C1421308D008D0B5E2B06180C15213005
:1006C6008D008D0B642B06188C1521308D008D0B3B
:1006D6006A2B06180C1621308D008D0B702B061810
:1006E6008C1621308D008D0B762B06180C172130B9
:1006F6008D008D0B7C2B06188C1721308D008D0BF1
:10070600822B21308D008D0B862B0C0883128B2BB0
:1007160083128E00851021308F008F0B902B0E0CCC
:10072600031C972B8514982B8510031083128E0CAF
:1007360021308F008F0B9D2B0E0C031CA42B8514D0
:10074600A52B8510031083128E0C21308F008F0B82
:10075600AA2B0E0C031CB12B8514B22B851003108B
:1007660083128E0C21308F008F0BB72B0E0C031CBF
:10077600BE2B8514BF2B8510031083128E0C2130DF
:100786008F008F0BC42B0E0C031CCB2B8514CC2B8C
:100796008510031083128E0C21308F008F0BD12B06
:1007A6000E0C031CD82B8514D92B8510031083122D
:1007B6008E0C21308F008F0BDE2B0E0C031CE52BCD
:1007C6008514E62B8510031083128E0C21308F00C2
:1007D6008F0BEB2B0E0C031CF22B8514F32B8510C1
:1007E600031083128E0C21308F008F0BF82B85148B
:0A07F60021308F008F0BFD2B08004F
:02400E00F93F78
:00000001FF
